BL51 BANKED LINKER/LOCATER V6.22                                                        09/21/2014  16:01:04  PAGE 1


BL51 BANKED LINKER/LOCATER V6.22, INVOKED BY:
C:\KEIL_C51\C51\BIN\BL51.EXE STARTUP.obj, main.obj, oled.obj TO OLED RAMSIZE (256)


MEMORY MODEL: SMALL


INPUT MODULES INCLUDED:
  STARTUP.obj (?C_STARTUP)
  main.obj (MAIN)
  oled.obj (OLED)
  C:\KEIL_C51\C51\LIB\C51S.LIB (?C?CLDOPTR)
  C:\KEIL_C51\C51\LIB\C51S.LIB (?C?IMUL)
  C:\KEIL_C51\C51\LIB\C51S.LIB (?C?UIDIV)


LINK MAP OF MODULE:  OLED (?C_STARTUP)


            TYPE    BASE      LENGTH    RELOCATION   SEGMENT NAME
            -----------------------------------------------------

            * * * * * * *   D A T A   M E M O R Y   * * * * * * *
            REG     0000H     0008H     ABSOLUTE     "REG BANK 0"
            DATA    0008H     000BH     UNIT         _DATA_GROUP_
            IDATA   0013H     0001H     UNIT         ?STACK

            * * * * * * *   C O D E   M E M O R Y   * * * * * * *
            CODE    0000H     0003H     ABSOLUTE     
            CODE    0003H     09D8H     UNIT         ?CO?OLED
            CODE    09DBH     0828H     UNIT         ?CO?MAIN
            CODE    1203H     00EEH     UNIT         ?PR?MAIN?MAIN
            CODE    12F1H     0094H     UNIT         ?C?LIB_CODE
            CODE    1385H     0092H     UNIT         ?PR?OLED_INIT?OLED
            CODE    1417H     0074H     UNIT         ?PR?_OLED_SHOWNUM?OLED
            CODE    148BH     0066H     UNIT         ?PR?_OLED_SHOWCHAR?OLED
            CODE    14F1H     0062H     UNIT         ?PR?_OLED_DRAWBMP?OLED
            CODE    1553H     0043H     UNIT         ?PR?_OLED_SHOWCHINESE?OLED
            CODE    1596H     003DH     UNIT         ?PR?_OLED_SHOWSTRING?OLED
            CODE    15D3H     0039H     UNIT         ?PR?_OLED_WR_BYTE?OLED
            CODE    160CH     0027H     UNIT         ?PR?OLED_CLEAR?OLED
            CODE    1633H     0020H     UNIT         ?PR?_OLED_SET_POS?OLED
            CODE    1653H     001AH     UNIT         ?PR?_DELAY_MS?OLED
            CODE    166DH     0018H     UNIT         ?PR?_OLED_POW?OLED
            CODE    1685H     0011H     UNIT         ?PR?OLED_DISPLAY_ON?OLED
            CODE    1696H     0011H     UNIT         ?PR?OLED_DISPLAY_OFF?OLED
            CODE    16A7H     000CH     UNIT         ?C_C51STARTUP



OVERLAY MAP OF MODULE:   OLED (?C_STARTUP)


SEGMENT                              DATA_GROUP 
  +--> CALLED SEGMENT              START    LENGTH
--------------------------------------------------
?C_C51STARTUP                      -----    -----
  +--> ?PR?MAIN?MAIN
BL51 BANKED LINKER/LOCATER V6.22                                                      09/21/2014  16:01:04  PAGE 2



?PR?MAIN?MAIN                      0008H    0001H
  +--> ?PR?OLED_INIT?OLED
  +--> ?PR?OLED_CLEAR?OLED
  +--> ?PR?_OLED_SHOWCHINESE?OLED
  +--> ?CO?MAIN
  +--> ?PR?_OLED_SHOWSTRING?OLED
  +--> ?PR?_OLED_SHOWCHAR?OLED
  +--> ?PR?_OLED_SHOWNUM?OLED
  +--> ?PR?_DELAY_MS?OLED
  +--> ?PR?_OLED_DRAWBMP?OLED

?PR?OLED_INIT?OLED                 -----    -----
  +--> ?PR?_DELAY_MS?OLED
  +--> ?PR?_OLED_WR_BYTE?OLED
  +--> ?PR?OLED_CLEAR?OLED
  +--> ?PR?_OLED_SET_POS?OLED

?PR?OLED_CLEAR?OLED                -----    -----
  +--> ?PR?_OLED_WR_BYTE?OLED

?PR?_OLED_SET_POS?OLED             -----    -----
  +--> ?PR?_OLED_WR_BYTE?OLED

?PR?_OLED_SHOWCHINESE?OLED         0009H    0001H
  +--> ?PR?_OLED_SET_POS?OLED
  +--> ?CO?OLED
  +--> ?PR?_OLED_WR_BYTE?OLED

?PR?_OLED_SHOWSTRING?OLED          0009H    0006H
  +--> ?PR?_OLED_SHOWCHAR?OLED

?PR?_OLED_SHOWCHAR?OLED            -----    -----
  +--> ?PR?_OLED_SET_POS?OLED
  +--> ?CO?OLED
  +--> ?PR?_OLED_WR_BYTE?OLED

?PR?_OLED_SHOWNUM?OLED             0009H    0009H
  +--> ?PR?_OLED_POW?OLED
  +--> ?PR?_OLED_SHOWCHAR?OLED

?PR?_OLED_POW?OLED                 0012H    0001H

?PR?_OLED_DRAWBMP?OLED             0009H    000AH
  +--> ?PR?_OLED_SET_POS?OLED
  +--> ?PR?_OLED_WR_BYTE?OLED



SYMBOL TABLE OF MODULE:  OLED (?C_STARTUP)

  VALUE           TYPE          NAME
  ----------------------------------

  -------         MODULE        ?C_STARTUP
  C:16A7H         SEGMENT       ?C_C51STARTUP
  I:0013H         SEGMENT       ?STACK
BL51 BANKED LINKER/LOCATER V6.22                                                      09/21/2014  16:01:04  PAGE 3


  C:0000H         PUBLIC        ?C_STARTUP
  D:00E0H         SYMBOL        ACC
  D:00F0H         SYMBOL        B
  D:0083H         SYMBOL        DPH
  D:0082H         SYMBOL        DPL
  N:0000H         SYMBOL        IBPSTACK
  N:0100H         SYMBOL        IBPSTACKTOP
  N:0080H         SYMBOL        IDATALEN
  C:16AAH         SYMBOL        IDATALOOP
  N:0000H         SYMBOL        PBPSTACK
  N:0100H         SYMBOL        PBPSTACKTOP
  N:0000H         SYMBOL        PDATALEN
  N:0000H         SYMBOL        PDATASTART
  N:0000H         SYMBOL        PPAGE
  N:0000H         SYMBOL        PPAGEENABLE
  D:00A0H         SYMBOL        PPAGE_SFR
  D:0081H         SYMBOL        SP
  C:16A7H         SYMBOL        STARTUP1
  N:0000H         SYMBOL        XBPSTACK
  N:0000H         SYMBOL        XBPSTACKTOP
  N:0000H         SYMBOL        XDATALEN
  N:0000H         SYMBOL        XDATASTART
  C:0000H         LINE#         126
  C:16A7H         LINE#         133
  C:16A9H         LINE#         134
  C:16AAH         LINE#         135
  C:16ABH         LINE#         136
  C:16ADH         LINE#         185
  C:16B0H         LINE#         196
  -------         ENDMOD        ?C_STARTUP

  -------         MODULE        MAIN
  C:0000H         SYMBOL        _ICE_DUMMY_
  D:0090H         PUBLIC        P1
  C:0A03H         PUBLIC        BMP1
  C:0E03H         PUBLIC        BMP2
  C:1203H         PUBLIC        main
  -------         PROC          MAIN
  -------         DO            
  D:0008H         SYMBOL        t
  -------         ENDDO         
  C:1203H         LINE#         17
  C:1203H         LINE#         18
  C:1203H         LINE#         21
  C:1206H         LINE#         22
  C:1209H         LINE#         38
  C:120CH         LINE#         39
  C:120CH         LINE#         40
  C:120CH         LINE#         41
  C:120FH         LINE#         42
  C:1216H         LINE#         43
  C:121FH         LINE#         44
  C:1228H         LINE#         45
  C:1231H         LINE#         46
  C:123AH         LINE#         47
  C:1243H         LINE#         48
  C:124CH         LINE#         49
BL51 BANKED LINKER/LOCATER V6.22                                                      09/21/2014  16:01:04  PAGE 4


  C:1259H         LINE#         51
  C:1266H         LINE#         52
  C:1273H         LINE#         53
  C:1280H         LINE#         54
  C:1289H         LINE#         55
  C:128BH         LINE#         56
  C:1295H         LINE#         57
  C:12A7H         LINE#         60
  C:12AEH         LINE#         61
  C:12B1H         LINE#         62
  C:12B8H         LINE#         63
  C:12CCH         LINE#         64
  C:12D3H         LINE#         65
  C:12E7H         LINE#         66
  C:12EEH         LINE#         67
  -------         ENDPROC       MAIN
  -------         ENDMOD        MAIN

  -------         MODULE        OLED
  C:0000H         SYMBOL        _ICE_DUMMY_
  C:1685H         PUBLIC        OLED_Display_On
  B:0090H.4       PUBLIC        OLED_RST
  D:0090H         PUBLIC        P1
  B:0090H.1       PUBLIC        OLED_DC
  C:1385H         PUBLIC        OLED_Init
  B:0090H.2       PUBLIC        OLED_CS
  C:1596H         PUBLIC        _OLED_ShowString
  C:15E4H         PUBLIC        _OLED_WR_Byte
  C:148BH         PUBLIC        _OLED_ShowChar
  C:0003H         PUBLIC        F6x8
  C:081BH         PUBLIC        Hzk
  B:0090H.0       PUBLIC        OLED_SDIN
  C:022BH         PUBLIC        F8X16
  C:1633H         PUBLIC        _OLED_Set_Pos
  C:1553H         PUBLIC        _OLED_ShowCHinese
  C:1653H         PUBLIC        _delay_ms
  C:1417H         PUBLIC        _OLED_ShowNum
  C:1696H         PUBLIC        OLED_Display_Off
  C:166DH         PUBLIC        _oled_pow
  B:0090H.3       PUBLIC        OLED_SCL
  C:160CH         PUBLIC        OLED_Clear
  C:14F1H         PUBLIC        _OLED_DrawBMP
  -------         PROC          _DELAY_MS
  D:0006H         SYMBOL        ms
  -------         DO            
  D:0004H         SYMBOL        a
  -------         ENDDO         
  C:1653H         LINE#         32
  C:1653H         LINE#         33
  C:1653H         LINE#         35
  C:1657H         LINE#         36
  C:1657H         LINE#         37
  C:165BH         LINE#         38
  C:1665H         LINE#         39
  C:166AH         LINE#         40
  C:166CH         LINE#         42
  -------         ENDPROC       _DELAY_MS
BL51 BANKED LINKER/LOCATER V6.22                                                      09/21/2014  16:01:04  PAGE 5


  C:15DDH         SYMBOL        L?0073
  -------         PROC          L?0072
  -------         ENDPROC       L?0072
  C:15DDH         SYMBOL        L?0073
  -------         PROC          _OLED_WR_BYTE
  D:0007H         SYMBOL        dat
  D:0005H         SYMBOL        cmd
  -------         DO            
  D:0006H         SYMBOL        i
  -------         ENDDO         
  C:15E4H         LINE#         64
  C:15E4H         LINE#         65
  C:15E4H         LINE#         67
  C:15E7H         LINE#         68
  C:15EBH         LINE#         70
  C:15EDH         LINE#         71
  C:15EFH         LINE#         72
  C:15F1H         LINE#         73
  C:15F1H         LINE#         74
  C:15F3H         LINE#         75
  C:15F7H         LINE#         76
  C:15F7H         LINE#         77
  C:15F9H         LINE#         78
  C:15FBH         LINE#         80
  C:15FDH         LINE#         81
  C:15FFH         LINE#         82
  C:1603H         LINE#         83
  C:1607H         LINE#         84
  C:1609H         LINE#         85
  C:160BH         LINE#         86
  -------         ENDPROC       _OLED_WR_BYTE
  -------         PROC          _OLED_SET_POS
  D:0004H         SYMBOL        x
  D:0005H         SYMBOL        y
  C:1633H         LINE#         88
  C:1635H         LINE#         89
  C:1635H         LINE#         90
  C:163EH         LINE#         91
  C:164AH         LINE#         92
  -------         ENDPROC       _OLED_SET_POS
  -------         PROC          OLED_DISPLAY_ON
  C:1685H         LINE#         95
  C:1685H         LINE#         96
  C:1685H         LINE#         97
  C:168CH         LINE#         98
  C:1691H         LINE#         99
  -------         ENDPROC       OLED_DISPLAY_ON
  -------         PROC          OLED_DISPLAY_OFF
  C:1696H         LINE#         102
  C:1696H         LINE#         103
  C:1696H         LINE#         104
  C:169DH         LINE#         105
  C:16A2H         LINE#         106
  -------         ENDPROC       OLED_DISPLAY_OFF
  -------         PROC          OLED_CLEAR
  -------         DO            
  D:0004H         SYMBOL        i
BL51 BANKED LINKER/LOCATER V6.22                                                      09/21/2014  16:01:04  PAGE 6


  D:0003H         SYMBOL        n
  -------         ENDDO         
  C:160CH         LINE#         109
  C:160CH         LINE#         110
  C:160CH         LINE#         112
  C:160EH         LINE#         113
  C:160EH         LINE#         114
  C:1617H         LINE#         115
  C:161CH         LINE#         116
  C:1621H         LINE#         117
  C:162EH         LINE#         118
  C:1632H         LINE#         119
  -------         ENDPROC       OLED_CLEAR
  -------         PROC          _OLED_SHOWCHAR
  D:0002H         SYMBOL        x
  D:0001H         SYMBOL        y
  D:0007H         SYMBOL        chr
  -------         DO            
  D:0003H         SYMBOL        c
  D:0004H         SYMBOL        i
  -------         ENDDO         
  C:148BH         LINE#         127
  C:1491H         LINE#         128
  C:1491H         LINE#         129
  C:1493H         LINE#         130
  C:1497H         LINE#         131
  C:14A1H         LINE#         132
  C:14A1H         LINE#         133
  C:14A1H         LINE#         134
  C:14A8H         LINE#         135
  C:14AAH         LINE#         136
  C:14C8H         LINE#         137
  C:14D0H         LINE#         138
  C:14D2H         LINE#         139
  -------         ENDPROC       _OLED_SHOWCHAR
  -------         PROC          _OLED_POW
  D:0012H         SYMBOL        m
  D:0001H         SYMBOL        n
  -------         DO            
  D:0006H         SYMBOL        result
  -------         ENDDO         
  C:166DH         LINE#         149
  C:1671H         LINE#         150
  C:1671H         LINE#         151
  C:1675H         LINE#         152
  C:1684H         LINE#         153
  C:1684H         LINE#         154
  -------         ENDPROC       _OLED_POW
  -------         PROC          _OLED_SHOWNUM
  D:0009H         SYMBOL        x
  D:000AH         SYMBOL        y
  D:000BH         SYMBOL        num
  D:000DH         SYMBOL        len
  D:000EH         SYMBOL        size2
  -------         DO            
  D:000FH         SYMBOL        t
  D:0010H         SYMBOL        temp
BL51 BANKED LINKER/LOCATER V6.22                                                      09/21/2014  16:01:04  PAGE 7


  D:0011H         SYMBOL        enshow
  -------         ENDDO         
  C:1417H         LINE#         161
  C:141FH         LINE#         162
  C:141FH         LINE#         164
  C:1422H         LINE#         165
  C:142BH         LINE#         166
  C:142BH         LINE#         167
  C:144DH         LINE#         168
  C:145BH         LINE#         169
  C:145BH         LINE#         170
  C:145FH         LINE#         171
  C:145FH         LINE#         172
  C:146CH         LINE#         173
  C:146EH         LINE#         174
  C:1471H         LINE#         176
  C:1471H         LINE#         177
  C:1486H         LINE#         178
  C:148AH         LINE#         179
  -------         ENDPROC       _OLED_SHOWNUM
  -------         PROC          _OLED_SHOWSTRING
  D:0009H         SYMBOL        x
  D:000AH         SYMBOL        y
  D:000BH         SYMBOL        chr
  -------         DO            
  D:000EH         SYMBOL        j
  -------         ENDDO         
  C:1596H         LINE#         181
  C:15A0H         LINE#         182
  C:15A0H         LINE#         183
  C:15A3H         LINE#         184
  C:15B5H         LINE#         185
  C:15BCH         LINE#         186
  C:15C2H         LINE#         187
  C:15CEH         LINE#         188
  C:15D0H         LINE#         189
  C:15D2H         LINE#         190
  -------         ENDPROC       _OLED_SHOWSTRING
  -------         PROC          _OLED_SHOWCHINESE
  D:0002H         SYMBOL        x
  D:0001H         SYMBOL        y
  D:0003H         SYMBOL        no
  -------         DO            
  D:0004H         SYMBOL        t
  D:0009H         SYMBOL        adder
  -------         ENDDO         
  C:1553H         LINE#         192
  C:1557H         LINE#         193
  C:1557H         LINE#         194
  C:155AH         LINE#         195
  C:155DH         LINE#         196
  C:155FH         LINE#         197
  C:155FH         LINE#         198
  C:156FH         LINE#         199
  C:1571H         LINE#         200
  C:1575H         LINE#         201
  C:157DH         LINE#         202
BL51 BANKED LINKER/LOCATER V6.22                                                      09/21/2014  16:01:04  PAGE 8


  C:157FH         LINE#         203
  C:157FH         LINE#         204
  C:158FH         LINE#         205
  C:1591H         LINE#         206
  C:1595H         LINE#         207
  -------         ENDPROC       _OLED_SHOWCHINESE
  -------         PROC          _OLED_DRAWBMP
  D:0009H         SYMBOL        x0
  D:0005H         SYMBOL        y0
  D:000BH         SYMBOL        x1
  D:000CH         SYMBOL        y1
  D:000DH         SYMBOL        BMP
  -------         DO            
  D:0010H         SYMBOL        j
  D:0004H         SYMBOL        x
  D:0012H         SYMBOL        y
  -------         ENDDO         
  C:14F1H         LINE#         209
  C:14F5H         LINE#         210
  C:14F5H         LINE#         211
  C:14FAH         LINE#         214
  C:150BH         LINE#         215
  C:1515H         LINE#         216
  C:151EH         LINE#         217
  C:151EH         LINE#         218
  C:1525H         LINE#         219
  C:152DH         LINE#         220
  C:152DH         LINE#         221
  C:154BH         LINE#         222
  C:154EH         LINE#         223
  C:1552H         LINE#         224
  -------         ENDPROC       _OLED_DRAWBMP
  -------         PROC          OLED_INIT
  C:1385H         LINE#         228
  C:1385H         LINE#         229
  C:1385H         LINE#         233
  C:1387H         LINE#         234
  C:138EH         LINE#         235
  C:1390H         LINE#         236
  C:1397H         LINE#         237
  C:1399H         LINE#         269
  C:13A0H         LINE#         270
  C:13A5H         LINE#         272
  C:13AAH         LINE#         274
  C:13AFH         LINE#         275
  C:13B4H         LINE#         277
  C:13B9H         LINE#         278
  C:13BEH         LINE#         280
  C:13C3H         LINE#         281
  C:13C8H         LINE#         283
  C:13CDH         LINE#         285
  C:13D2H         LINE#         287
  C:13D7H         LINE#         289
  C:13DCH         LINE#         290
  C:13E1H         LINE#         292
  C:13E6H         LINE#         293
  C:13EBH         LINE#         295
BL51 BANKED LINKER/LOCATER V6.22                                                      09/21/2014  16:01:04  PAGE 9


  C:13F0H         LINE#         296
  C:13F5H         LINE#         298
  C:13FAH         LINE#         299
  C:13FFH         LINE#         301
  C:1404H         LINE#         303
  C:1409H         LINE#         306
  C:140EH         LINE#         307
  C:1411H         LINE#         308
  -------         ENDPROC       OLED_INIT
  -------         ENDMOD        OLED

  -------         MODULE        ?C?CLDOPTR
  C:12F1H         PUBLIC        ?C?CLDOPTR
  -------         ENDMOD        ?C?CLDOPTR

  -------         MODULE        ?C?IMUL
  C:131EH         PUBLIC        ?C?IMUL
  -------         ENDMOD        ?C?IMUL

  -------         MODULE        ?C?UIDIV
  C:1330H         PUBLIC        ?C?UIDIV
  -------         ENDMOD        ?C?UIDIV

*** WARNING L16: UNCALLED SEGMENT, IGNORED FOR OVERLAY PROCESS
    SEGMENT: ?PR?OLED_DISPLAY_ON?OLED

*** WARNING L16: UNCALLED SEGMENT, IGNORED FOR OVERLAY PROCESS
    SEGMENT: ?PR?OLED_DISPLAY_OFF?OLED

Program Size: data=20.0 xdata=0 code=5811
LINK/LOCATE RUN COMPLETE.  2 WARNING(S),  0 ERROR(S)
